:020000040000FA
:0608000035EF2AF01200A2
:02080600FEFFF3
:06080800C4EF17F012001E
:02080E00C250D6
:08081000020B01E0010E1200D1
:06081800E2EF0EF01200F9
:02081E000600D2
:1008200022550000E3020000090000001E550000F0
:10083000F0020000040000001C550000F40200005B
:100840000200000003550000E5010000190000004F
:1008500006080000FE01000002000000F85400003D
:08086000CE0200000B000000B5
:0808680070EC09F0FB0EDBCF80
:10087000F3FFDB06F35000090AE0BEEC09F0FA0EC4
:1008800029EC0AF0F3E12C1CF1E1010E01D0000E7D
:100890009FEF09F070EC09F03B0EE12402E3E16800
:1008A000E652E16E010EDB6A020EDB6AF90EDBCF67
:1008B000F6FFFA0EDBCFF7FFFB0EDBCFF8FF0800E9
:1008C000F550DF6EDF5002E1C5EF08F0250EDF5C6A
:1008D00002E0B8EF08F0030EDB6A040EDB6A050ED7
:1008E000DB6A060EDB6A070EDB6AD8EC08F02D0E19
:1008F000DF5C0CE02B0EDF5C09E0200EDF5C06E025
:10090000230EDF5C03E0300EDF5C1AE1DF50300ABB
:1009100014E0130A0FE0030A0AE00B0A05E0060AD6
:10092000E4E1030EDB80E1D7030EDB82DED7030EAA
:10093000DB84DBD7030EDB86D8D7030EDB88D5D765
:100940002A0EDF5C1BE1D4EC08F022EC09F010E089
:10095000030EDB801D681E68130EDBCF22F0140E21
:10096000DBCF23F083EC25F0040E1BC0DBFF03D0AC
:10097000130E0BEC09F0D8EC08F00BD0090EDB6A73
:1009800079EC09F003E0EDEC09F0FAD7090E0BEC75
:1009900009F0030EDBB0DB982E0EDF5C1BE1D8EC18
:1009A00008F02A0EDF5C0BE1D4EC08F022EC09F031
:1009B00003E1130E5DEC09F0D8EC08F00BD0090E42
:1009C000DB6A79EC09F003E0EDEC09F0FAD7090EE7
:1009D0005DEC09F0680EDF5C07E1D8EC08F0680E0A
:1009E000DF5C1DE1030E18D0740EDF5C17E07A0E99
:1009F000DF5C14E0480EDF5C06E0540EDF5C03E0D1
:100A00005A0EDF5C02E1020E07D06C0EDF5C03E0E1
:100A10006A0EDF5C04E1010EB0EC09F0C9DBDF50C7
:100A20006E0A01E181D31E0A01E192D1200A01E19F
:100A30008FD13F0A01E149D11A0A01E146D10D0ADD
:100A400001E143D1200A01E140D13A0A01E13DD15F
:100A5000200A01E13AD1260A01E135D10D0A01E16E
:100A600032D11A0A01E1D9D0200A4AE0300A1FE047
:100A7000460A0EE0250A01E085D3D950F90FE96E48
:100A8000FF0EDA20EA6E010EEE5E000EEE5AEE5A0E
:100A9000BEEC09F0250EE66E95DB03E12C1C01E1AE
:100AA0006BD3BAEC09F001E26DD3DB2A6BD3080EED
:100AB000DB6A040EDB50010806E2040EDB0482EC64
:100AC00009F0DB508BDB080EDB5009E0030EDB5036
:100AD000010B05E172DB01E04FD3080EDB6A64DB3A
:100AE000EFCFDFFF32EC0AF003E12C1C01E144D32D
:100AF000BAEC09F001E3DB2A60DB01E143D33CD32C
:100B0000070EDB5002080FE1FEEC09F0030EC5EC06
:100B100009F00E0EEECFDBFF0F0EEECFDBFF100E57
:100B2000EECFDBFF20D0F70EDBCF2EF0F80EDBCFC1
:100B30002FF0020E2E5E000E2F5AF70E2EC0DBFF96
:100B4000F80E2FC0DBFF2EC0E9FF2FC0EAFFB5EC87
:100B500009F02D6A0E0E2BC0DBFF0F0E2CC0DBFF41
:100B6000100E2DC0DBFF0E0EDBCFE6FF0F0EDBCF2E
:100B7000E6FF100EDBCFE6FF80EC27F0E552E552F2
:100B8000E552130E1CC0DBFF140E1DC0DBFF060E6A
:100B9000DB5005E0130EF9EC09F001E26ADB1DEC15
:100BA0000AF002E2130E37DBE0EC09F006E0040E77
:100BB000F9EC09F002E2050E2EDB030EDBB005D0E6
:100BC000FCDA01E0D9D2080EDB6A090EDB6A0E0EF0
:100BD000DBCFF6FF0F0EDBCFF7FF100EDBCFF8FFFA
:100BE0000800F550DF6EDF5014E023EC0AF011E24C
:100BF00032EC0AF003E12C1C01E1BED2BBDB01E3C5
:100C0000DB2A090EDB2AD9500E0FE96E000ECBDB72
:100C1000E7D7D3DA01E1B6D2AFD2C6DA110EEECF02
:100C2000DBFF120EEDCFDBFF110EDBCFE6FF120E66
:100C3000DBCFE6FF72EC27F0E552E552130EF3CF5F
:100C4000DBFF140EF4CFDBFF060EDB5004E0130EC7
:100C5000D0DB01E20EDB1DEC0AF002E2130EDBDA60
:100C6000AFDB05E0040EC5DB02E2050ED4DA030EAD
:100C7000DBB005D0A2DA01E07FD2080EDB6A090EF4
:100C8000DB6A110EDBCFE9FF120EDBCFEAFFEFCFFD
:100C9000DFFFDF5014E0D7DB12E2E4DB03E12C1CC2
:100CA00001E16AD267DB01E3DB2A090EDB2A110EC0
:100CB000DB2ADBCFE9FF120EE8E3DB2AE6D77DDA99
:100CC00001E160D259D2030EDB8E070EDB0410E186
:100CD00095DB040E5ADB0A0EEECFDBFF0B0EEECFD8
:100CE000DBFF0C0EEECFDBFF0D0EEECFDBFF6CD08B
:100CF000070EDB5003082CE1030EDBAE0DD0B2DA99
:100D0000020E76DAEFCF2BF02C6A2D6A2E6A2BAE0C
:100D100039D02C682D6835D0F70EDBCF2CF0F80ECB
:100D2000DBCF2DF0020E2C5E000E2D5AF70E2CC0DC
:100D3000DBFFF80E2DC0DBFF2CC0E9FF2DC0EAFF62
:100D4000EFCF2BF00A0E2BC0DBFF0B0EDB6A38D087
:100D5000070EDB50020809E1030EDBAE04D059DBBD
:100D60002DAE10D00ED055DB0DD0030EDBAE12D061
:100D700079DA020E3DDAF9DA2D6A2E6A2CAE02D04B
:100D80002D682E68E2DA0C0E2DC0DBFF0D0E2EC092
:100D9000DBFF1AD0F70EDBCF2DF0F80EDBCF2EF0F5
:100DA000020E2D5E000E2E5AF70E2DC0DBFFF80E40
:100DB0002EC0DBFF2DC0E9FF2EC0EAFFD6DAC5DA70
:100DC0000C0EDB6A0D0EDB6A060EDB5005E1010E30
:100DD000F36E050EF3CFDBFF150EDB6A160EDB6A32
:100DE000D950370F2B6E000EDA202C6E390E2BC027
:100DF000DBFF3A0E2CC0DBFF380EDB6A080EDB6A25
:100E00000A0EAEDADF50780A12E0200A10E0280A53
:100E10000CE0200A0AE03F0A06E00D0A02E0200A80
:100E200008E1020E05D0080E03D0080EDF26100ED2
:100E300097DA030EDBBE02D0DB92DB94DB50800B33
:100E400026E08ADA030EEB50000AE8AE02D0D89012
:100E500008D0000EEE5C000EEE58000EEE58000EAC
:100E6000EE5815E211DA206821682268236878ECD0
:100E700028F00A0E17C0DBFF0B0E18C0DBFF0C0EAC
:100E800019C0DBFF0D0E1AC0DBFF2D0E08D0030EBC
:100E9000DBA202D02B0E03D0DBA408D0200EF36E11
:100EA000170EF3CFDBFF150EDB2A02D0170EDB6A1D
:100EB000050EDB5003E1B5D901E189D0DC0E2B6EC4
:100EC000540E2C6E000E2D6E070EDBCF2EF02F6A07
:100ED000306A316A2EC020F02FC021F030C022F0DD
:100EE00031C023F0D1D9A1EC29F02B501724F36E97
:100EF0002C501820F46E2D501920F86EF4CFF7FF07
:100F0000F3CFF6FF0800090EF5CFDBFF580EDF5CCC
:100F10000FE1610EF36E090E79D90AE3200E2B6EF4
:100F2000090EDBCFE7FF2B50E75E090EE7CFDBFFB3
:100F3000070EDBCF2BF02C6A2D6A2E6A0DDA2BC040
:100F400020F02CC021F02DC022F02EC023F0EECFD7
:100F50001BF0EECF1CF0EECF1DF0EFCF1EF0A1EC9A
:100F600029F01EC0EDFF1DC0EDFF1CC0EDFF1BC032
:100F7000EFFF390EDBCFE9FFDB063A0EDBCFEAFFEE
:100F800001E2DB06090EDBCFEFFF150EDB2A49D9A4
:100F900095E1030EDBA61DD06F0EDF5C06E1BFD925
:100FA00018E3150EDB2859DA14D0780EDF5C09E05F
:100FB000580EDF5C06E0620EDF5C03E0420EDF5C91
:100FC00008E1020EF36E160EF3CFDBFF02D0150E12
:100FD000DB6A030EDB50100B0EE0040EDBCF2BF0B0
:100FE000050EDB50D8802B5406E2060EDB5003E1E1
:100FF000040EDB5032DA93D90AE2050EDBCFE7FFAD
:10100000150EDB50E75E050EE7CFDBFF02D0050EC5
:10101000DB6A040EDBCF2BF0160E43D9D8802B549D
:1010200014E2160EDBCFE6FF150EDBCFE6FF040E53
:10103000DBCFE6FF050EDB50E552E75CE552D880DA
:10104000E754E552D880E7545DD9030EDB50010B1D
:101050000BE1080EDB5008E0B0D801E08DD0080E9F
:10106000DB50BCD8080EDB6A170EDB5007E086D9D0
:10107000170EEFD903E12C1C01E17ED0160EDB50D8
:1010800016E07CD9300EE66E9DD802E12C1C74E08F
:1010900075D9DFCFE6FF36EC28F0E552E552E55290
:1010A000F4CF2CF00001F31C02E12C1C65E0050ECE
:1010B000DBCF2BF0160EDB50D8802B5409E2050E47
:1010C000DBCFE7FF160EDB50E75E050EE7CFDBFF59
:1010D000300EE66E050EC9D94FE1390EDB2ADBCFA3
:1010E000E9FF3A0E01E3DB2ADBCFEAFF090EEFCF7F
:1010F000DBFFDB500EE042D9090EABD902E12C1C1C
:101100003BE0390EDB2ADBCFE9FF3A0EEDE3DB2AC9
:10111000EBD753D831E1160EDBCFE6FF080EC1D86E
:10112000E552E7245BD82ED0070EDB50030A1CE003
:10113000010A14E0030A07E079D9DBCFEEFF020EC3
:10114000DBCFEDFF1FD0F3D8306A2EAE02D02F6870
:1011500030682AD8BAD830C0EEFF14D0E8D82EBEF6
:101160002F6822D8B2D80ED061D9DBCFEFFF0AD0DA
:1011700079D905E12C1C03E1F368F46810D0FAD8A2
:1011800001E3DB2A77D95FEF04F0010EDBCF2BF010
:10119000020EDBCF2CF02BC0F3FF2CC0F4FFD9CF15
:1011A000E1FFDACFE2FFCBD029D9020EC5EF09F07B
:1011B00061D90800F550DF6E1200200EE66E080EB1
:1011C00035EF0AF036EC28F0E552E552E552F3CF60
:1011D0002BF0F4CF2CF00001F31C12002B6E2C6AC4
:1011E000D950010F4DD92B50EE262C50ED22120074
:1011F0002F5E000E305AF70E2FC0DBFFF80E30C006
:10120000DBFF2FC0E9FF30C0EAFF1200DBCFF4FFA5
:10121000F350F45C1200DB50E76E040EE7CFDBFF07
:1012200012000A0EDBCF2BF00B0EDBCF2CF00C0ED6
:10123000DBCF2DF00D0EDBCF2EF02B502C102D1010
:101240002E101200130EEECFDBFF140EEDCFDBFFDE
:10125000130EDBCF2BF0140EDBCF2CF00001800E31
:101260002C141200F70EDBCF2FF0F80EDBCF30F08E
:101270001200050EDB50E66ED950130F01D9E5526E
:10128000E750EE6EED6A12000A0EDBCF1BF00B0E7C
:10129000DBCF1CF00C0EDBCF1DF00D0EDBCF1EF0F4
:1012A0001200DBCFE6FF150EDBCFE6FF050EDB50AD
:1012B000E552E724E552E7241200DB50CED8010EB8
:1012C000F36E060EF3CFDBFF1200EE50EFCFEAFF16
:1012D000E96E2DC0EEFF2EC0EEFF2FC0EEFF120014
:1012E000D9CFE6FFDACFE6FFE1CFD9FFE2CFDAFFD1
:1012F0001200DFCFE6FFE66A23EC2AF0E552E55262
:10130000F3501200E76E080EE7CFDBFF1200EECFBE
:101310002BF0EECF2CF0EFCF2DF02E6A1200050E41
:10132000DBCF2BF0150EDB50D8802B541200010EB2
:10133000DBCF2DF0020EDBCF2EF02F6A1200E5522C
:10134000E5CFDAFFE7CFD9FF12000A0E2BC0DBFF93
:101350000B0E2CC0DBFF1200D9500A0F40EF0AF031
:10136000F36E070EF3CFDBFF1200EECF2BF0EFCFC3
:101370002CF01200010EDB2A020E1200FC0EDBCF55
:10138000E6FFFD0EDBCFE6FF12002B5E000E2C5AAF
:10139000F70E2BC0DBFFF80E2CC0DBFF2BC0E9FFE4
:1013A0002CC0EAFF1200DA20EA6EEF2AEECFF6FF39
:1013B000000EEF22EECFF7FFEF22EECFF8FF120084
:1013C000040EDBCFE6FF130EDB50E552E75C9ADF3D
:1013D000DB5004DF060EDB501200090EDB500A0D55
:1013E000F350DF24D00FE76E090EE7CFDBFFD8EF15
:1013F00008F0DB50F36E050E06EF09F0F70EDBCFB9
:101400002BF0F80EDBCF2CF01200DFCFE6FFE2EF7F
:1014100008F028DF030EECDE87EF09F034EC04F06F
:10142000E552E552E552E55200091200BDDEEE50EC
:10143000EFCFEAFFE96E010E1200130EDB50F36EE0
:10144000040E06EF09F0040EDB50F36E090E06EFF2
:1014500009F0DBCFE6FFE2EF08F0E76E050EE7CF1D
:10146000DBFF12008BDF05EF0AF0DBCFE6FF86DF44
:101470000EEF0AF0D950F90FE96EFF0ED3EF09F025
:0A148000E96E000EDA20EA6E120099
:06148A00D9CFE6FFE1CF1F
:10149000D9FF020EE126DE6ADD6A0201F451F51180
:1014A00003E1F36AF46A3AD0F407000EF55BF4C284
:1014B0002BF0F5C22CF0090E2C02F3CF2CF02B02EE
:1014C000F3CF2BF0F4502C26CB0E2B26010E2C2222
:1014D0002BC0DEFF2CC0DDFFDECFE9FFDDCFEAFF52
:1014E000040EE926000EEA22FD0EDBCFEEFFFE0E13
:1014F000DBCFEDFFFC0EDBCFE6FFDECFE6FFDDCF7F
:10150000E6FF12D8E552E552E552DECF2BF0DDCFF3
:101510002CF02BC0F3FF2CC0F4FF00D0D9CFE1FF9B
:10152000E552E7CFD9FF1200D9CFE6FFE1CFD9FFCF
:10153000020EE126FD0EDBCFDEFFDBCFDDFFDECFCF
:10154000E9FFDDCFEAFFEE6AEE6AEE6AEE6ADECF11
:10155000E9FFDDCFEAFF060EE926000EEA22EF6A78
:10156000DECFE9FFDDCFEAFF070EE926000EEA2213
:10157000EF6ADECFE9FFDDCFEAFF080EE926000EB5
:10158000EA22FC0EDBCFEFFFD9CFE1FFE552E7CF38
:10159000D9FF1200D9CFE6FFE1CFD9FF030EE12634
:1015A000FD0EDBCF1DF0FE0EDBCF1EF0DE521DC0A8
:1015B000DEFF1EC0DDFFDD52FC0EDB50030BE76ECD
:1015C000FC0EE7CFDBFFDBCFE6FF010EDBCFE9FF51
:1015D000020EDBCFEAFF080EE926000EEA22EF50EA
:1015E000040DF350E552E710DF6EDF50030A1BE0F5
:1015F000040A19E00F0A17E0040A15E00E0A07E0D2
:10160000040A05E00F0A03E0040A01E018D0010E05
:10161000DBCFE9FF020EDBCFEAFF060EE926000E64
:10162000EA22EF2A0CD0010EDBCFE9FF020EDBCF5E
:10163000EAFF060EE926000EEA22EF0600D0010EB0
:10164000DBCFE9FF020EDBCFEAFF080EE926000E32
:10165000EA22FC0EDBCFEFFFD9CFE1FFE552E7CF67
:10166000D9FF1200D9CFE6FFE1CFD9FF040EE12662
:10167000FD0EDBCF1DF0FE0EDBCF1EF0020E1DC0F7
:10168000DBFF030E1EC0DBFF020EDBCFE9FF030E04
:10169000DBCFEAFF060EE926000EEA22EFCFDFFFDE
:1016A000020EDBCFE9FF030EDBCFEAFF070EE926D0
:1016B000000EEA22EF50DF5CE76E010EE7CFDBFFA2
:1016C000DBCF2BF02C6A2D6A2E6A2BAE03D02C6850
:1016D0002D682E68020EDBCFE9FF030EDBCFEAFF99
:1016E0002B50EE262C50EE222D50EE222E50EE22C4
:1016F000020EDBCFE9FF030EDBCFEAFF070EE92680
:10170000000EEA22DFCFEFFF010EDB5000D0D9CF71
:10171000E1FFE552E7CFD9FF1200D9CFE6FFE1CFD5
:10172000D9FF060EE126FD0EDBCFDEFFDBCFDDFFAE
:10173000DECFE9FFDDCFEAFF040EE926000EEA2244
:10174000EECF2FF0EFCF30F0316A326A30AE02D0F8
:1017500031683268DECFE9FFDDCFEAFFEECF2BF054
:10176000EECF2CF0EECF2DF0EFCF2EF02BC01BF0F4
:101770002CC01CF02DC01DF02EC01EF02FC020F07C
:1017800030C021F031C022F032C023F078EC28F0D4
:10179000020E17C0DBFF030E18C0DBFF040E19C0DA
:1017A000DBFF050E1AC0DBFF020EDBCF1BF0030EC2
:1017B000DBCF1CF0040EDBCF1DF0050EDBCF1EF0DF
:1017C000E80E206E030E216E226A236A4FEC25F08C
:1017D000020E1BC0DBFF030E1CC0DBFF040E1DC08E
:1017E000DBFF050E1EC0DBFF020EDBCF2BF0030E6E
:1017F000DBCF2CF0040EDBCF2DF0050EDBCF2EF06F
:101800002BC01BF02CC01CF02DC01DF02EC01EF0F4
:1018100000D0D9CFE1FFE552E7CFD9FF1200D9CFF1
:10182000E6FFE1CFD9FFFB0EDBCFE1F1FC0EDBCF12
:10183000E2F1FD0EDBCFE3F1FE0EDBCFE4F1F90EBA
:10184000DBCFDDF1FA0EDBCFDEF1F70EDBCFDFF120
:10185000F80EDBCFE0F1DD0E2B6E010E2C6E2BC0EF
:10186000F3FF2CC0F4FF00D0E552E7CFD9FF120000
:10187000D9CFE6FFE1CFD9FF1C0EE126FD0EDBCF6D
:10188000DEFFDBCFDDFFDECFE9FFDDCFEAFFEE508D
:10189000EFCFEAFFE96E0C0EEECFDBFF0D0EEECFC1
:1018A000DBFF0E0EEECFDBFF0F0EEECFDBFF0C0EDD
:1018B000DBCF1BF00D0EDBCF1CF00E0EDBCF1DF0CF
:1018C0000F0EDBCF1EF0100E206E270E216E226A47
:1018D000236A78EC28F0140E17C0DBFF150E18C031
:1018E000DBFF160E19C0DBFF170E1AC0DBFFDECFC1
:1018F000E9FFDDCFEAFFEE50EFCFEAFFE96E040E1D
:10190000E926000EEA22EECF2BF0EFCF2CF02D6A65
:101910002E6A2CAE02D02D682E682BC020F02CC071
:1019200021F02DC022F02EC023F0140EDBCF1BF0CF
:10193000150EDBCF1CF0160EDBCF1DF0170EDBCF24
:101940001EF04FEC25F0140E1BC0DBFF150E1CC063
:10195000DBFF160E1DC0DBFF170E1EC0DBFFDECF48
:10196000E9FFDDCFEAFF020EE926000EEA22EE5083
:10197000EFCFEAFFE96E100EEECFDBFF110EEECFD8
:10198000DBFF120EEECFDBFF130EEECFDBFF100EF0
:10199000DBCF1BF0110EDBCF1CF0120EDBCF1DF0E6
:1019A000130EDBCF1EF0100E206E270E216E226A62
:1019B000236A78EC28F0180E17C0DBFF190E18C048
:1019C000DBFF1A0E19C0DBFF1B0E1AC0DBFFDECFD8
:1019D000E9FFDDCFEAFF020EE926000EEA22EE5013
:1019E000EFCFEAFFE96E040EE926000EEA22EECF01
:1019F0002BF0EFCF2CF02D6A2E6A2CAE02D02D6882
:101A00002E682BC020F02CC021F02DC022F02EC05B
:101A100023F0180EDBCF1BF0190EDBCF1CF01A0ED3
:101A2000DBCF1DF01B0EDBCF1EF04FEC25F0180EA8
:101A30001BC0DBFF190E1CC0DBFF1A0E1DC0DBFF35
:101A40001B0E1EC0DBFF140EDBCF2FF0150EDBCFFD
:101A500030F0160EDBCF31F0170EDBCF32F0D9505D
:101A6000180FE96EDACFEAFFEE502F5C2B6EEE50C6
:101A700030582C6EEE5031582D6EEE5032582E6E7E
:101A8000040E2BC0DBFF050E2CC0DBFF060E2DC0A5
:101A9000DBFF070E2EC0DBFFDECFE9FFDDCFEAFF65
:101AA000040EE926000EEA22EECF1BF0EECF1CF06A
:101AB000EECF1DF0EFCF1EF0640E206E216A226A79
:101AC000236A4FEC25F0080E1BC0DBFF090E1CC07B
:101AD000DBFF0A0E1DC0DBFF0B0E1EC0DBFF040E7A
:101AE000DBCF1CF0050EDBCF1DF0060EDBCF1EF0AA
:101AF000070EDBCF1FF0000E1F18E8AE02D01F3418
:101B000009D0000ED8801C54000E1D54000E1E5427
:101B1000000E1F540DE2040EDBCF2BF0050EDBCFC1
:101B20002CF0060EDBCF2DF0070EDBCF2EF02ED0E3
:101B3000040EDBCF1BF0050EDBCF1CF0060EDBCF57
:101B40001DF0070EDBCF1EF0206821682268236895
:101B500078EC28F0000E1A18E8AE02D01A3409D03A
:101B6000A00ED8801754860E1854010E1954000E7A
:101B70001A5402E3000E01D0010E2B6E2C6A2D6A5E
:101B80002E6A2BAE03D02C682D682E682B502C109B
:101B90002D102E1070E0040EDBCF1BF0050EDBCFF6
:101BA0001CF0060EDBCF1DF0070EDBCF1EF0640E1F
:101BB000206E216A226A236A78EC28F0020E17C090
:101BC000DBFF030E18C0DBFF020EDBCF2BF0030E92
:101BD000DBCF2CF02D6A2E6A2CAE02D02D682E6839
:101BE0002BC01BF02CC01CF02DC01DF02EC01EF011
:101BF000080EDBCF20F0090EDBCF21F00A0EDBCF81
:101C000022F00B0EDBCF23F04FEC25F0020E1BC0B1
:101C1000DBFF030E1CC0DBFF020EDBCF2BF0030E3D
:101C2000DBCF2CF0B40E2C02F3CF2CF02B02F3CF31
:101C30002BF0F4502C26D8902B362C36020E2BC0CD
:101C4000DBFF030E2CC0DBFF3A0E2B6E010E2C6E59
:101C5000020EDBCF1DF0030EDBCF1EF02BC022F0F7
:101C60002CC023F029EC25F0020E1DC0DBFF030E73
:101C70001EC0DBFF77D0040EDBCF1BF0050EDBCFE1
:101C80001CF0060EDBCF1DF0070EDBCF1EF0B40EEE
:101C9000206E216A226A236A78EC28F017C01BF0B4
:101CA00018C01CF019C01DF01AC01EF0020E206EE4
:101CB000216A226A236A78EC28F0020E17C0DBFF43
:101CC000030E18C0DBFF3A0E2B6E010E2C6E020EB7
:101CD000DBCF1DF0030EDBCF1EF02BC022F02CC09B
:101CE00023F029EC25F0020E1DC0DBFF030E1EC001
:101CF000DBFF640E1D6E1E6A020EDBCF22F0030EA8
:101D0000DBCF23F083EC25F0020E1BC0DBFF030EBC
:101D10001CC0DBFF020EDBCF2BF0030EDBCF2CF061
:101D20002D6A2E6A2CAE02D02D682E682BC01BF0B7
:101D30002CC01CF02DC01DF02EC01EF0080EDBCFF5
:101D400020F0090EDBCF21F00A0EDBCF22F00B0EC4
:101D5000DBCF23F04FEC25F0020E1BC0DBFF030EA0
:101D60001CC0DBFF010EE76E020EDBCF2BF0030E73
:101D7000DBCF2CF0E7502B26000E2C22020E226E19
:101D8000236A2BC01DF02CC01EF029EC25F01DC0CD
:101D90002BF01EC02CF0020E2BC0DBFF030E2CC05C
:101DA000DBFF020EDBCF2BF0030EDBCF2CF02BC0C2
:101DB000F3FF2CC0F4FF00D0D9CFE1FFE552E7CF0D
:041DC000D9FF120035
:0C1DC400D8CFE4FFE0CFE4FFE46EDACFFC
:101DD000E4FFE2CFDAFFE9CFE4FFEACFE4FFF3CF9D
:101DE000E4FFF4CFE4FFE652D9CFE6FFE1CFD9FF1D
:101DF000020EE1269E50200B06E09D50200B03E0D2
:101E00003EEC21F049D0A450200B06E0A350200B5B
:101E100003E05DEC21F040D09E50100B06E09D5099
:101E2000100B03E07CEC21F037D0A450100B06E03F
:101E3000A350100B03E094EC21F02ED0F050020BD5
:101E400007E0F050100B04E0F092E6EC25F024D00F
:101E5000F050040B07E0F050200B04E0F09422EC6B
:101E600026F01AD0F250010B17E0F250080B14E0E4
:101E70008150DF6EF290DF500201EB19E76E010E28
:101E8000E7CFDBFFDFCFEBF2DBA800D0DBAA00D08F
:101E9000DBAC00D0DBAE00D0D9CFE1FFE552E7CF1D
:101EA000D9FFE552E5CFF4FFE5CFF3FFE5CFEAFF39
:101EB000E5CFE9FFE5CFDAFFE550E5CFE0FFE5CF7D
:101EC000D8FF1000D9CFE6FFE1CFD9FF130EE126EE
:101ED000040EDB6A050EDB6A080EDB6A02017F0E68
:101EE0008B6F8BC28AF28BC289F28BC288F28BC253
:101EF00087F28BC286F28BC285F28BC284F2936F1B
:101F000093C292F293C291F293C290F293C28FF273
:101F100093C28EF293C28DF293C28CF28C928D9208
:101F20008C908D908C968D968C948D948C9A8D9AA5
:101F30008C988D988C9E91908C9C8D9C060EDB6A63
:101F400088B6DB8082B0DB8288B8DB8488BADB8627
:101F500088BCDB8888BEDB8ADB503F0AE76E060E52
:101F6000E7CFDBFFDB50100A1DE0180A15E0290A55
:101F70000DE0280A0BE0080A03E0070EDB6A18D020
:101F8000010EF36E070EF3CFDBFF12D0010EF36EDE
:101F9000070EF3CFDBFF0CD0080EF36E070EF3CF66
:101FA000DBFF06D0090EF36E070EF3CFDBFF00D088
:101FB0000201A1AD8FD30201C0A18BD3070EDB506C
:101FC000E76E120EE7CFDBFFA00EE66E020EE66EA6
:101FD000D5EC18F0E552E552BAEC25F0090E1BC01D
:101FE000DBFF0A0E1CC0DBFF0B0E1DC0DBFF0C0E5F
:101FF0001EC0DBFFF6EC25F00D0E1BC0DBFF0E0E46
:102000001CC0DBFF0F0E1DC0DBFF100E1EC0DBFF70
:10201000020EDB6A030EDB6ADE6ADD6A060EDBCFC8
:102020008BF2E66AE66AE66AE66AD950090FE96E5B
:10203000DACFEAFFEECFE6FFEECFE6FFEECFE6FF28
:10204000EFCFE6FFC8EC21F0F56E080EE15EF5502B
:102050001BC08CF2D9500D0FE96EDACFEAFFEECF3C
:10206000E6FFEECFE6FFEECFE6FFEFCFE6FFE66A54
:10207000E66AE66AE66AC8EC21F0F56E080EE15EF3
:10208000F5501BC08DF2870EE66E84EC23F0E5520E
:10209000F3CF2BF0F4CF2CF0D8902C322B32D890F9
:1020A0002C322B322BC08EF2070EDBCF8FF2DB509F
:1020B000090A01E18CD2010A01E17CD20F0A01E197
:1020C000D4D1020A01E130D1060A01E1AAD0010A05
:1020D00001E192D0060A01E18FD0020A01E18CD021
:1020E000070A07E0020EDB6A030EDB6ADE6ADD6ABE
:1020F000A3D2D9500D0FE96EDACFEAFFEECFE6FF9B
:10210000EECFE6FFEECFE6FFEFCFE6FFD950090FA7
:10211000E96EDACFEAFFEECFE6FFEECFE6FFEECFD5
:10212000E6FFEFCFE6FF56EC22F0F56E080EE15E1B
:10213000F550000E1E18E8AE02D01E3409D0000E75
:10214000D8801B54000E1C54000E1D54000E1E544B
:102150000AE2DE6ADD6A7F0EF36E020EF3CFDBFF6A
:10216000030EDB6A07D07F0EDE6EDD6A020EDB6ACD
:10217000030EDB6AD9500D0FE96EDACFEAFFEECF1E
:10218000E6FFEECFE6FFEECFE6FFEFCFE6FFD9505A
:10219000090FE96EDACFEAFFEECFE6FFEECFE6FFFA
:1021A000EECFE6FFEFCFE6FFC8EC21F0F56E080EAC
:1021B000E15EF5501E50000AE8AE02D0D89008D07B
:1021C000C20E1B5C010E1C58000E1D58000E1E583E
:1021D00012E3E80EE66E030EE66ED950040FE66ECB
:1021E000000EDA20E66E7EEC24F0E552E552E55270
:1021F000E552120EDB2A20D2020EDB6A030EDB6AE6
:10220000DE6ADD6AD950040FE66E000EDA20E66E53
:10221000D5EC24F0E552E552000902E0120EDB2A6B
:102220000BD2060EDBAA10D0A60EF36E110EF3CF62
:10223000DBFF810EDE6EDD687F0EF36E020EF3CFE4
:10224000DBFF030EDB6A0FD05A0EF36E110EF3CFD5
:10225000DBFF7F0EDE6EDD6A810EF36E020EF3CFC2
:10226000DBFF030EDB68110EDBCF2BF02C6A2D6A2F
:102270002E6A2BAE03D02C682D682E682BC0E6FF8B
:102280002CC0E6FF2DC0E6FF2EC0E6FFD9500D0F93
:10229000E96EDACFEAFFEECFE6FFEECFE6FFEECF54
:1022A000E6FFEFCFE6FFD950090FE96EDACFEAFF7C
:1022B000EECFE6FFEECFE6FFEECFE6FFEFCFE6FF95
:1022C00056EC22F0F56E080EE15EF550E552E7CFD0
:1022D0002EF0E552E7CF2DF0E552E7CF2CF0E55296
:1022E000E7CF2BF01E502E18E8AE02D02E3408D0C7
:1022F0002B501B5C2C501C582D501D582E501E5816
:1023000012E3E80EE66E030EE66ED950040FE66E99
:10231000000EDA20E66E7EEC24F0E552E552E5523E
:10232000E552120EDB2A88D1110EDBCF2BF02C6A7E
:102330002D6A2E6A2BAE03D02C682D682E682BC018
:10234000E6FF2CC0E6FF2DC0E6FF2EC0E6FFD95009
:102350000D0FE96EDACFEAFFEECFE6FFEECFE6FF34
:10236000EECFE6FFEFCFE6FFD950090FE96EDACFE7
:10237000EAFFEECFE6FFEECFE6FFEECFE6FFEFCFD0
:10238000E6FF56EC22F0F56E080EE15EF550E552E0
:10239000E7CF2EF0E552E7CF2DF0E552E7CF2CF056
:1023A000E552E7CF2BF02E501E18E8AE02D01E34B7
:1023B00008D01B502B5C1C502C581D502D581E5003
:1023C0002E580AE2DE6ADD6A7F0EF36E020EF3CF4C
:1023D000DBFF030EDB6A07D07F0EDE6EDD6A020EC6
:1023E000DB6A030EDB6AD9500D0FE96EDACFEAFF24
:1023F000EECFE6FFEECFE6FFEECFE6FFEFCFE6FF54
:10240000D950090FE96EDACFEAFFEECFE6FFEECF43
:10241000E6FFEECFE6FFEFCFE6FFC8EC21F0F56E6A
:10242000080EE15EF5501E50000AE8AE02D0D890CA
:1024300008D0340E1B5C020E1C58000E1D58000EF6
:102440001E5812E3E80EE66E030EE66ED950040F36
:10245000E66E000EDA20E66E7EEC24F0E552E552E0
:10246000E552E552120EDB2AE7D0110EDBCF2BF03E
:102470002C6A2D6A2E6A2BAE03D02C682D682E682C
:102480002BC0E6FF2CC0E6FF2DC0E6FF2EC0E6FF06
:10249000D9500D0FE96EDACFEAFFEECFE6FFEECFAF
:1024A000E6FFEECFE6FFEFCFE6FFD950090FE96E6A
:1024B000DACFEAFFEECFE6FFEECFE6FFEECFE6FFA4
:1024C000EFCFE6FF56EC22F0F56E080EE15EF55018
:1024D000E552E7CF2EF0E552E7CF2DF0E552E7CFFA
:1024E0002CF0E552E7CF2BF02E501E18E8AE02D0AC
:1024F0001E3408D01B502B5C1C502C581D502D58DE
:102500001E502E5808E2810EDE6EDD68020EDB6A78
:10251000030EDB6A09D0DE6ADD6A810EF36E020EFD
:10252000F3CFDBFF030EDB68D9500D0FE96EDACF76
:10253000EAFFEECFE6FFEECFE6FFEECFE6FFEFCF0E
:10254000E6FFD950090FE96EDACFEAFFEECFE6FFDA
:10255000EECFE6FFEECFE6FFEFCFE6FFC8EC21F0CF
:10256000F56E080EE15EF550000E1E18E8AE02D0C2
:102570001E3409D0C20ED8801B54010E1C54000E0C
:102580001D54000E1E5415E3E80EE66E030EE66EB3
:10259000D950040FE66E000EDA20E66E7EEC24F0D1
:1025A000E552E552E552E552040EF36E120EF3CFFA
:1025B000DBFF42D07F0EF36E020EF3CFDBFF030E84
:1025C000DB6A020EDBCFDEFFDBCFDDFF35D0020E94
:1025D000DB6A030EDB6ADE6ADD6A020EE66EFD0E62
:1025E000E66E050EE66E870EE66E84EC23F0E5528D
:1025F000F3CF2DF0F4CF2EF0D8902E322D32D8908C
:102600002E322D322D50E66E7D0EE66E880EE66E71
:10261000020EE66EEFEC27F0F56E070EE15EF55068
:10262000F3CF2BF0F4CF2CF0010E2B1801E12C503E
:1026300002E1120EDB6A00D0120EDB50E76E070ECD
:10264000E7CFDBFF080EDBCFF3FFDB2AF3500208F6
:1026500002E2080EDB6ADECFE6FFDDCFE6FF7BECB1
:1026600029F0E552E5520201856F846F020EDBCF3F
:102670002BF0030EDBCF2CF02B6C2C1E000E2C222B
:102680002BC0E6FF2CC0E6FF7BEC29F0E552E552BB
:102690000201876F866F93C2E6FF92C2E6FF91C286
:1026A000E6FF90C2E6FFE2EC1FF0E552E552E5528C
:1026B000E5528150040B02E0919001D091808C9EF4
:1026C000800EE66E020EE66EEEEC18F0E552E55274
:1026D00000D06ED4D9CFE1FFE552E7CFD9FF120089
:0226E0001200E6
:0E26E200F00EE66E79EC23F0E552938A9388B1
:1026F0009386938499829980938E938C9A849A82FC
:10270000998699849A8A9A8894809A869A8E9A8CC5
:1027100002017F0E8B6F8BC28AF28BC289F28BC251
:1027200088F28BC287F28BC286F28BC285F28BC293
:1027300084F2936F93C292F293C291F293C290F299
:1027400093C28FF293C28EF293C28DF293C28CF237
:102750005EEC20F077EC20F00101010EE56FB0ECAB
:1027600025F0800EE66E020EE66EEEEC18F0E552F5
:10277000E552F40EE66E530EE66E000EE66EA5EC24
:1027800027F0E552E552E55275EF18F0D9CFE6FF94
:10279000E1CFD9FFFD0EDBCFE9FFFE0EDBCFEAFF75
:1027A000EF50F36EFC0EDB50F35C14E0FD0EDBCF5C
:1027B000E9FFFE0EDBCFEAFFEF040CE1FD0EDBCFFD
:1027C000E9FFFE0EDBCFEAFFFC0EDBCFEFFF010ED1
:1027D0000CD00BD0FD0EDBCFE9FFFE0EDBCFEAFF06
:1027E000FC0EDBCFEFFF000E00D0E552E7CFD9FFA4
:1027F0001200D9CFE6FFE1CFD9FF120EE126870EF6
:10280000E66E84EC23F0E552F3CF2BF0F4CF2CF0FE
:10281000D8902C322B32D8902C322B322BC08EF207
:10282000A00EE66E020EE66ED5EC18F0E552E5520B
:102830000201D851D82B0E0801E2D86BD551030AFA
:1028400043E0070A2DE0010A17E0070A01E050D033
:102850000201A351200B01E0010EE66ED00EE66EE0
:10286000020EE66E93DFE552E552E552010803E100
:102870000201050ED56F3CD00201A351200B01E0EF
:10288000010EE66ED00EE66E020EE66E7FDFE552BA
:10289000E552E552000903E10201040ED56F28D08C
:1028A0000201A351200B01E0010EE66ED00EE66E90
:1028B000020EE66E6BDFE552E552E552010803E1D8
:1028C0000201030ED56F14D00201A351200B01E0C9
:1028D000010EE66ED00EE66E020EE66E57DFE55292
:1028E000E552E552000903E10201020ED56F00D066
:1028F0000201D5A303D08D808C9002D08D908C8066
:10290000D651030A01E183D0050A69E0010A4FE0CC
:10291000030A35E0010A1BE0070A01E090D08D921E
:102920008C828D948C840201A351100B01E0010E66
:10293000E66ED10EE66E020EE66E28DFE552E55237
:10294000E552000903E00201050ED66F78D08D82B2
:102950008C928D948C840201A351100B01E0010E26
:10296000E66ED10EE66E020EE66E10DFE552E5521F
:10297000E552000903E10201040ED66F60D08D829A
:102980008C928D948C840201A351100B01E0010EF6
:10299000E66ED10EE66E020EE66EF8DEE552E55208
:1029A000E552010803E10201070ED66F48D08D827F
:1029B0008C928D948C840201A351100B01E0010EC6
:1029C000E66ED10EE66E020EE66EE0DEE552E552F0
:1029D000E552000903E10201060ED66F30D08D8268
:1029E0008C928D848C940201A351100B01E0010E96
:1029F000E66ED10EE66E020EE66EC8DEE552E552D8
:102A0000E552010803E10201030ED66F18D08D9242
:102A10008C828D948C840201A351100B01E0010E75
:102A2000E66ED10EE66E020EE66EB0DEE552E552BF
:102A3000E552000903E10201020ED66F00D0020147
:102A4000D751050A4FE0010A34E0070A16E0010AEF
:102A500001E068D00201A351200B01E0010EE66EF7
:102A6000CE0EE66E020EE66E91DEE552E552E552BE
:102A7000000902E08D968C8655D00201010E8A6F06
:102A80008AC289F20201A351200B01E0010EE66E19
:102A9000CE0EE66E020EE66E79DEE552E552E552A6
:102AA000000903E19350400B03E00201040ED76FCD
:102AB00039D002017F0E8A6F8AC289F20201A351C6
:102AC000200B01E0010EE66ECE0EE66E020EE66E03
:102AD0005DDEE552E552E552000903E10201050E13
:102AE000D76F20D002018A698AC289F293AE02D0E0
:102AF0007F0E896F99A002D07F0E8A6F0201A351C9
:102B0000200B01E0010EE66ECE0EE66E020EE66EC2
:102B10003DDEE552E552E552010803E10201030EF4
:102B2000D76F00D0AAC2E6FF8CEC29F0E552080E60
:102B3000F3CFDBFF090EF4CFDBFFA6C2E6FF8CEC80
:102B400029F0E5520A0EF3CFDBFF0B0EF4CFDBFFCB
:102B5000A7C2E6FF8CEC29F0E5520C0EF3CFDBFFA9
:102B60000D0EF4CFDBFFAEC2E6FF0A0EDBCFE6FFB1
:102B70000B0EDBCFE6FFA7EC26F0E552E552E5525F
:102B80000A0EF3CFDBFF0B0EF4CFDBFFAEC2E6FF86
:102B9000080EDBCFE6FF090EDBCFE6FFA7EC26F041
:102BA000E552E552E552080EF3CFDBFF090EF4CFF4
:102BB000DBFFAEC2E6FF0C0EDBCFE6FF0D0EDBCF78
:102BC000E6FFA7EC26F0E552E552E5520C0EF3CFF6
:102BD000DBFF0D0EF4CFDBFF0201D451030A43E00B
:102BE000070A2DE0010A17E0070A01E050D00201B0
:102BF000A251020B01E0010EE66ECF0EE66E020E50
:102C0000E66EC4DDE552E552E552010803E102013A
:102C1000050ED46F3CD00201A251020B01E0010E5F
:102C2000E66ECF0EE66E020EE66EB0DDE552E552C0
:102C3000E552000903E10201040ED46F28D002011D
:102C4000A251020B01E0010EE66ECF0EE66E020EFF
:102C5000E66E9CDDE552E552E552010803E1020112
:102C6000030ED46F14D00201A251020B01E0010E39
:102C7000E66ECF0EE66E020EE66E88DDE552E55298
:102C8000E552000903E10201020ED46F00D00201F7
:102C9000D4A329D0080EDBCF2DF0090EDBCF2EF008
:102CA0000A0EDB502D242B6E0B0EDB502E202C6ECB
:102CB0000E0E2BC0DBFF0F0E2CC0DBFF0A0EDBCF8E
:102CC0002DF00B0EDBCF2EF0080EDB502D5C2B6EA3
:102CD000090EDB502E582C6E100E2BC0DBFF110E90
:102CE0002CC0DBFF18D00C0EDBCF1DF00D0EDBCFA0
:102CF0001EF00E0E1DC0DBFF0F0E1EC0DBFF0A0E06
:102D0000DBCF1DF00B0EDBCF1EF0100E1DC0DBFF66
:102D1000110E1EC0DBFFD351030A43E0070A2DE06A
:102D2000010A17E0070A01E050D00201A351020B8B
:102D300001E0010EE66ED20EE66E020EE66E26DDB4
:102D4000E552E552E552010803E10201050ED36F99
:102D50003CD00201A351020B01E0010EE66ED20E3F
:102D6000E66E020EE66E12DDE552E552E55200090E
:102D700003E10201040ED36F28D00201A351020B1C
:102D800001E0010EE66ED20EE66E020EE66EFEDC8D
:102D9000E552E552E552010803E10201030ED36F4B
:102DA00014D00201A351020B01E0010EE66ED20E17
:102DB000E66E020EE66EEADCE552E552E5520009E7
:102DC00003E10201020ED36F00D00201D3A303D0AE
:102DD000A9C288F204D0A9C28AF2A9C289F20E0E51
:102DE000DBCF2DF00F0EDBCF2EF02E3404E32D5071
:102DF0008108FF0E2E5407E20E0EDBCF2BF00F0ED4
:102E0000DBCF2CF003D0810E2B6E2C680E0E2BC066
:102E1000DBFF0F0E2CC0DBFF0E0EDBCF2DF00F0EF5
:102E2000DBCF2EF0D8902E5004E67F0E2D5C000EE6
:102E30002E5807E20E0EDBCF2BF00F0EDBCF2CF05F
:102E400003D07F0E2B6E2C6A0E0E2BC0DBFF0F0EF5
:102E50002CC0DBFF100EDBCF2DF0110EDBCF2EF0E0
:102E60002E3404E32D508108FF0E2E5407E2100E7D
:102E7000DBCF2BF0110EDBCF2CF003D0810E2B6EAD
:102E80002C68100E2BC0DBFF110E2CC0DBFF100EC8
:102E9000DBCF2DF0110EDBCF2EF0D8902E5004E6B4
:102EA0007F0E2D5C000E2E5807E2100EDBCF2BF0AC
:102EB000110EDBCF2CF003D07F0E2B6E2C6A100E80
:102EC0002BC0DBFF110E2CC0DBFF0E0EDBCFE6FFAD
:102ED0000F0EDBCFE6FF7BEC29F0E552E552020155
:102EE000856F846F100EDBCF2BF0110EDBCF2CF033
:102EF0002B6C2C1E000E2C222BC0E6FF2CC0E6FFF4
:102F00007BEC29F0E552E5520201876F866F815014
:102F1000800B02E0919001D091808C9EBAEC25F05C
:102F20001BC0DEFF1CC0DEFF1DC0DEFF1EC0DDFFBC
:102F3000DD52DD52F6EC25F0040E1BC0DBFF050E62
:102F40001CC0DBFF060E1DC0DBFF070E1EC0DBFF33
:102F500093C2E6FF92C2E6FF91C2E6FF90C2E6FF8F
:102F6000E2EC1FF0E552E552E552E552800EE66EC6
:102F7000020EE66EEEEC18F0E552E552D9CFE1FF15
:082F8000E552E7CFD9FF120072
:082F8800D8CFE4FFE0CFE4FF25
:102F9000E46EDACFE4FFE2CFDAFFE9CFE4FFEACF75
:102FA000E4FFE652F2A202D0A5D802D09EB6D1D854
:102FB000E552E5CFEAFFE5CFE9FFE5CFDAFFE550DF
:102FC000E5CFE0FFE5CFD8FF1000E66A010EE66E20
:102FD000050EE66EE4EC28F0E552E552E5521200EB
:102FE000070EB46E000E886E876E866E856E846ED8
:102FF000836E826E816E806E916E906E8F6E8E6E1D
:103000008D6E8C6E8B6E8A6E896E2F0E926E9368AB
:103010009C0E946E956A966A9768040E986E0E0ED2
:103020009A6E9968C16AF19EB0989C8EA26A9F6A56
:10303000A06A9D6AA36AA56AC8DF9F86D08E9E9605
:103040009D869382F06AF288F09EF098F192F09A51
:10305000F16AF28CF28E1200D9CFE6FFE1CFD9FFF0
:10306000E652BEDF0201C097C0990201840ECC6F08
:10307000020ECD6FDF6A100EDF5C0AE2DF50EA6AF3
:10308000CC25E96ECD51EA227F0EEF6EDF2AF3D711
:1030900002019D6B010E9E6FC20E9F6F0201C085E3
:1030A0000201A26BA36B0201806B826B836B010E2A
:1030B000D56E320ED76ECF0ED66ED59E800EE66ED2
:1030C000020EE66E8BD8E552E5520201C093800EE7
:1030D000E66E020EE66E82D8E552E5520201C0931A
:1030E000E552E552E7CFD9FF1200828280889492A0
:1030F00092981200F2920201200EC86F9F86020180
:10310000C0A906D00201E00EC56F000EC66F05D043
:103110000201C00EC56F000EC66F0201C0A1C079CA
:10312000C0A706D00201800EC36F000EC46F05D089
:103130000201A00EC36F000EC46FC9CFC9F2C3C293
:10314000E9FFC4C2EAFFC32B000EC423EF50C96ECF
:1031500012009E96C9CFC9F20201C851000823E2AD
:10316000C5C2E9FFC6C2EAFFC52B000EC623C9C20D
:10317000EFFFC3C2E9FFC4C2EAFFC32BC423EFCFF2
:10318000C9F2C9C2C9FFC807C8510CE10201020E49
:103190009E6F0201C093C081320ED76ECF0ED66EE5
:1031A000F294D58E01D0C96A1200D9CFE6FFE1CFE3
:1031B000D9FF0201C0A10ED0FD0EDBCFE6FFFE0E4F
:1031C000DBCFE6FF4EEC1FF0E552E5529D96020183
:1031D000C0919D86E552E7CFD9FF1200D9CFE6FF17
:1031E000E1CFD9FF0201C0B332D0FD0EDBCFE9FF42
:1031F000FE0EDBCFEAFF1E0EE926000EEA22EF509C
:10320000020809E1FD0EDBCFE6FFFE0EDBCFE6FF95
:1032100069D8E552E552FD0EDBCFE9FFFE0EDBCFAC
:10322000EAFF150EE926000EEA22EF9EFD0EDBCF27
:10323000E6FFFE0EDBCFE6FFBCEC1EF0E552E552EA
:103240009D960201C077C0839D8602019D2BE552A9
:10325000E7CFD9FF12009D960201C0919D86120012
:10326000D9CFE6FFE1CFD9FF0001166BD950FD0F92
:10327000E96EFF0EDA20EA6E010EEE1801E1ED5064
:1032800002E1168101D0BA6AD950FB0FE96EFF0E38
:10329000DA20EA6E010EEE1801E1ED5002E116832C
:1032A00001D0B76AD950F90FE96EFF0EDA20EA6E45
:1032B000010EEE1801E1ED5002E1168501D0736AAE
:1032C000D950F70FE96EFF0EDA20EA6E010EEE1804
:1032D00001E1ED5002E1168701D0706AE552E7CFB7
:1032E000D9FF1200D9CFE6FFE1CFD9FFFD0EDBCF2A
:1032F000E9FFFE0EDBCFEAFF1C0EE926000EEA22F4
:10330000EF6AFD0EDBCFE9FFFE0EDBCFEAFF170E03
:10331000E926000EEA22EF6AC6AE0ED0C69EFD0E6A
:10332000DBCFE9FFFE0EDBCFEAFF170EE926000E2A
:10333000EA22010EEF6E22D0F150800B10E0F25025
:10334000080B0DE0FD0EDBCFE9FFFE0EDBCFEAFF41
:10335000170EE926000EEA22020EEF6E0FD0F0A63D
:103360000DD0909EFD0EDBCFE9FFFE0EDBCFEAFF16
:10337000170EE926000EEA22030EEF6E250EC61484
:10338000250819E0FD0EDBCFE9FFFE0EDBCFEAFFDB
:103390001C0EE926000EEA22010EEF6EFD0EDBCFB9
:1033A000E9FFFE0EDBCFEAFF170EE926000EEA2248
:1033B000C6CFEFFF80D1C55019E0FD0EDBCFE9FF8E
:1033C000FE0EDBCFEAFF1C0EE926000EEA22020EFB
:1033D000EF6EFD0EDBCFE9FFFE0EDBCFEAFF170E2F
:1033E000E926000EEA22C5CFEFFF65D1D0BE19D085
:1033F000FD0EDBCFE9FFFE0EDBCFEAFF1C0EE92658
:10340000000EEA22030EEF6EFD0EDBCFE9FFFE0E8B
:10341000DBCFEAFF170EE926000EEA22D0CFEFFF3E
:103420004AD19DB619D0FD0EDBCFE9FFFE0EDBCFF2
:10343000EAFF1C0EE926000EEA22040EEF6EFD0ED6
:10344000DBCFE9FFFE0EDBCFEAFF170EE926000E09
:10345000EA229DCFEFFF2FD19C5019E0FD0EDBCF6C
:10346000E9FFFE0EDBCFEAFF1C0EE926000EEA2282
:10347000050EEF6EFD0EDBCFE9FFFE0EDBCFEAFFA0
:10348000170EE926000EEA229CCFEFFF14D1080E9A
:103490009F5C19E0FD0EDBCFE9FFFE0EDBCFEAFFFC
:1034A0001C0EE926000EEA22060EEF6EFD0EDBCFA3
:1034B000E9FFFE0EDBCFEAFF170EE926000EEA2237
:1034C0009FCFEFFFF8D0A25019E0FD0EDBCFE9FF50
:1034D000FE0EDBCFEAFF1C0EE926000EEA22070EE5
:1034E000EF6EFD0EDBCFE9FFFE0EDBCFEAFF170E1E
:1034F000E926000EEA22A2CFEFFFDDD0A55019E0A9
:10350000FD0EDBCFE9FFFE0EDBCFEAFF1C0EE92646
:10351000000EEA22080EEF6EFD0EDBCFE9FFFE0E75
:10352000DBCFEAFF170EE926000EEA22A5CFEFFF58
:10353000C2D0100EF214100819E0FD0EDBCFE9FF27
:10354000FE0EDBCFEAFF1C0EE926000EEA22090E72
:10355000EF6EFD0EDBCFE9FFFE0EDBCFEAFF170EAD
:10356000E926000EEA22F2CFEFFFA5D0470EF114B4
:1035700019E0FD0EDBCFE9FFFE0EDBCFEAFF1C0EEC
:10358000E926000EEA220A0EEF6EFD0EDBCFE9FF00
:10359000FE0EDBCFEAFF170EE926000EEA22F1CF7E
:1035A000EFFF89D0C00EF01419E0FD0EDBCFE9FF6C
:1035B000FE0EDBCFEAFF1C0EE926000EEA220B0E00
:1035C000EF6EFD0EDBCFE9FFFE0EDBCFEAFF170E3D
:1035D000E926000EEA22F0CFEFFF6DD092A819D0B5
:1035E000FD0EDBCFE9FFFE0EDBCFEAFF1C0EE92666
:1035F000000EEA220C0EEF6EFD0EDBCFE9FFFE0E91
:10360000DBCFEAFF170EE926000EEA2292CFEFFF8A
:1036100052D093B019D0FD0EDBCFE9FFFE0EDBCF09
:10362000EAFF1C0EE926000EEA220D0EEF6EFD0EDB
:10363000DBCFE9FFFE0EDBCFEAFF170EE926000E17
:10364000EA2293CFEFFF37D03E0E94141C0819E006
:10365000FD0EDBCFE9FFFE0EDBCFEAFF1C0EE926F5
:10366000000EEA220E0EEF6EFD0EDBCFE9FFFE0E1E
:10367000DBCFEAFF170EE926000EEA2294CFEFFF18
:103680001AD097BE18D0FD0EDBCFE9FFFE0EDBCFC0
:10369000EAFF1C0EE926000EEA220F0EEF6EFD0E69
:1036A000DBCFE9FFFE0EDBCFEAFF170EE926000EA7
:0E36B000EA2297CFEFFFE552E7CFD9FF1200D5
:0236BE00D9CF62
:1036C000E6FFE1CFD9FFF29CFD0EDBCFE9FFFE0E56
:1036D000DBCFEAFFEE52EF6AFD0EDBCFE9FFFE0E15
:1036E000DBCFEAFF540EE926000EEA22EF6AF28CE5
:1036F000E552E7CFD9FF1200D9CFE6FFE1CFD9FFDE
:10370000E6520101AE0E5D6F0F0E5E6FAD0E5F6F84
:103710000F0E606F010E086F080EE66E010EE66E6A
:10372000CEDFE552E55201016E0EB66F0F0EB76F98
:103730006D0EB86F0F0EB96F020E616F610EE66EFF
:10374000010EE66EBCDFE552E552150EE66E7C0E0C
:10375000E66E49EC29F0E552E5529F989F9A949CB9
:10376000948EAE50DF6EAE50DF6E9E9A150EE66EF2
:103770007C0EE66E17EC29F0E552E552A59AA59865
:10378000989298846E50DF6E6E50DF6EA49A01019D
:10379000BA6BE552E552E7CFD9FF1200D9CFE6FF69
:1037A000E1CFD9FFFD0EDBCFE9FFFE0EDBCFEAFF55
:1037B000EF0402E19D8801D0A388E552E7CFD9FF4D
:1037C0001200D9CFE6FFE1CFD9FFD950FD0FE96E46
:1037D000FF0EDA20EA6EEE50ED100AE19EA807D047
:1037E000080EE66E010EE66ED9DFE552E55209D00D
:1037F000A4A807D0610EE66E010EE66ECFDFE5529B
:10380000E552E552E7CFD9FF1200D9CFE6FFE1CF6D
:10381000D9FFD950FD0FE96EFF0EDA20EA6EEE50A7
:10382000ED1005E1ABB2AB98AB889D8A04D06BB2CA
:103830006B986B88A38AE552E7CFD9FF1200D9CFE6
:10384000E6FFE1CFD9FFFD0EDBCFE9FFFE0EDBCFB8
:10385000EAFFEF0403E19E989D9802D0A498A398F4
:10386000E552E7CFD9FF1200D9CFE6FFE1CFD9FF6C
:10387000FD0EDBCFE9FFFE0EDBCFEAFFEE52EF508D
:103880000AE1FD0EDBCFE6FFFE0EDBCFE6FFD7DF62
:10389000E552E5522FD0FD0EDBCFE9FFFE0EDBCF68
:1038A000EAFF020EE926000EEA22EECFF3FFEDCF8B
:1038B000F4FFEE2AEF22F3CFE9FFF4CFEAFFEF5057
:1038C000E66EFD0EDBCFE9FFFE0EDBCFEAFF570E03
:1038D000E926000EEA22EE50EFCFEAFFE96EE5524C
:1038E000E750EF6EFD0EDBCFE9FFFE0EDBCFEAFF08
:1038F000EE52EF06E552E7CFD9FF1200D9CFE6FF2F
:10390000E1CFD9FFE65201010651060A4FE0030A52
:1039100041E0010A37E0070A2DE0010A1EE0030A30
:103920000CE0010A02E0066B4FD0066BFE0EDB5086
:10393000C90802E1010E066F47D0066B079BFE0E19
:10394000DB50170802E1079D05D0FE0EDB5018087A
:1039500001E1078D020E066F37D0FE0EDBCF02F1BC
:10396000DBCF98F20251800B01E0010EBA6F030E1B
:10397000066F2AD0FE0EDBCF03F1DBCF99F2040EE7
:10398000066F22D0FE0EDBCF04F1DBCF9AF2050EDC
:10399000066F1AD0FE0EDBCF05F1DBCF9BF207AD31
:1039A00003D0060E066F01D0066B0ED00251032520
:1039B00004250525DF6EDF1CF36EFE0EDB50F35C85
:1039C00001E1078B066B00D0E552E552E7CFD9FF46
:1039D00012009EAA0AD09E9A5DC1E9FF5EC1EAFF6D
:1039E000EF50E66E8BDFE55216D09EA807D0080E8A
:1039F000E66E010EE66E38DFE552E552A4AA02D06B
:103A0000A49A09D0A4A807D0610EE66E010EE66E56
:103A10002BDFE552E55212007CEF1BF0D9CFE6FF19
:103A2000E1CFD9FF590E1D6E1E6AFD0EDBCF22F0CD
:103A3000FE0EDBCF23F083EC25F01BC0C7F11CC0CA
:103A4000C8F1080E0101C727010EC823F29CC7C1A7
:103A5000E9FFC8C1EAFF020EE926000EEA22FB0ECA
:103A6000DBCFEEFFFC0EDBCFEDFFC7C1E9FFC8C126
:103A7000EAFFEE52F90EDBCFEFFFF28CFD0EDBCF4B
:103A8000E6FFFE0EDBCFE6FF9CDEE552E552E55297
:103A9000E7CFD9FF1200D9CFE6FFE1CFD9FFFD0E66
:103AA000DBCFE9FFFE0EDBCFEAFF590EEA02F3CFD0
:103AB000EAFFE902F3CFE9FFF450EA26080EE9260F
:103AC000010EEA22EE52EF50000801E2E8D7F80EAC
:103AD000DBCF2BF0F90EDBCF2CF02C3404E22B5093
:103AE0005008000E2C5407E2500EF36EF80EF3CF80
:103AF000DBFFF90EDB6AFA0EDBCFE6FFFB0EDBCF56
:103B0000E6FFFC0EDBCFE6FFBB0EE66E010EE66EB7
:103B100059EC27F0F56E050EE15EF550F80EDBCF9F
:103B2000E6FFF90EDBCFE6FFBB0EE66E010EE66E9A
:103B3000FD0EDBCFE6FFFE0EDBCFE6FF6FDFF56E9F
:103B4000060EE15EF550000E00D0E552E7CFD9FF3A
:103B50001200D9CFE6FFE1CFD9FF590E1D6E1E6AC4
:103B6000FD0EDBCF22F0FE0EDBCF23F083EC25F041
:103B70001BC0C9F11CC0CAF1080E0101C927010E02
:103B8000CA23C9C1E9FFCAC1EAFF570EE926000EE0
:103B9000EA22EE50EFCFEAFFE96EFB0EDBCFEFFF3C
:103BA000D950FD0FE96EFF0EDA20EA6EEE50ED10EF
:103BB00003E19EA8FED702D0A4A8FED7E552E7CF26
:103BC000D9FF1200D9CFE6FFE1CFD9FF010109519A
:103BD000000801E2FBD75C515C2BEA6A0C0FE96E2E
:103BE000010EEA22FE0EDBCFEFFFDB500D0803E0F3
:103BF000500E5C5D0FE3F29C0C0E0A6F010E0B6F12
:103C00005CC109F1F28C5C6B000EE66EE66AD9DDF0
:103C1000E552E552E552E7CFD9FF1200010107ADA9
:103C200002D0010E02D0000E00D01200D9CFE6FF64
:103C3000E1CFD9FF020EE126010EDB6A010107ADDB
:103C400004D007BB02D0DB5068D0090EF36EFE0E25
:103C5000DBCFF4FFF350F45C13E2FE0EDB042B6EBB
:103C6000010E2B5204E0E846FE0B2B06FCE1DF6E52
:103C7000DF5001010515E76E010EE7CFDBFF4BD0EA
:103C8000110EF36EFE0EDBCFF4FFF350F45C14E282
:103C9000FE0EDB50F70F2B6E010E2B5204E0E846B0
:103CA000FE0B2B06FCE1DF6EDF5001010415E76E11
:103CB000010EE7CFDBFF2FD0190EF36EFE0EDBCF28
:103CC000F4FFF350F45C14E2FE0EDB50EF0F2B6EAA
:103CD000010E2B5204E0E846FE0B2B06FCE1DF6EE2
:103CE000DF5001010315E76E010EE7CFDBFF13D0B4
:103CF000FE0EDB50E70F2B6E010E2B5204E0E84660
:103D0000FE0B2B06FCE1DF6EDF5001010215E76EB2
:103D1000010EE7CFDBFFDB5000D0D9CFE1FFE5524A
:063D2000E7CFD9FF1200FD
:0A3D2600000EE96EEA6E0400A0EC46
:103D30001EF0EA2A080EEA5CD8A496EF1EF01200E4
:103D4000EF6AE93EA0EF1EF01200FF0EE3CF09F08C
:103D500009380F0B060FD8B2070F2A0FAD6ED8EC3B
:103D600022F009500F0B060FD8B2070F2A0FAD6EC5
:103D7000D8EC22F0000C1200EACF04F0E9CF05F0F5
:103D8000FF0EE3CFEAFFFE0EE3CFE9FFC0A741D06D
:103D9000EECFA0F0EECFA1F0EECFA2F0EECFA3F0E9
:103DA000EECFA4F0EECFA5F0EECFA6F0EECFA7F0C9
:103DB000EECFA8F0EECFA9F0EECFAAF0EECFABF0A9
:103DC000EECFACF0EECFADF0EECFAEF0EECFAFF089
:103DD000EECFB0F0EECFB1F0EECFB2F0EECFB3F069
:103DE000EECFB4F0EECFB5F0EECFB6F0EECFB7F049
:103DF000EECFB8F0EECFB9F0EECFBAF0EECFBBF029
:103E0000EECFBCF0EECFBDF0EECFBEF0EECFBFF008
:103E100040D0EECF80F0EECF81F0EECF82F0EECF4B
:103E200083F0EECF84F0EECF85F0EECF86F0EECFCC
:103E300087F0EECF88F0EECF89F0EECF8AF0EECFAC
:103E40008BF0EECF8CF0EECF8DF0EECF8EF0EECF8C
:103E50008FF0EECF90F0EECF91F0EECF92F0EECF6C
:103E600093F0EECF94F0EECF95F0EECF96F0EECF4C
:103E700097F0EECF98F0EECF99F0EECF9AF0EECF2C
:103E80009BF0EECF9CF0EECF9DF0EECF9EF0EECF0C
:103E90009FF004C0EAFF05C0E9FF1200C0A11200B4
:103EA000EACF04F0E9CF05F0FF0EE3CFEAFFFE0E04
:103EB000E3CFE9FFC0A941D0C0C0EEFFC1C0EEFF13
:103EC000C2C0EEFFC3C0EEFFC4C0EEFFC5C0EEFF30
:103ED000C6C0EEFFC7C0EEFFC8C0EEFFC9C0EEFF10
:103EE000CAC0EEFFCBC0EEFFCCC0EEFFCDC0EEFFF0
:103EF000CEC0EEFFCFC0EEFFD0C0EEFFD1C0EEFFD0
:103F0000D2C0EEFFD3C0EEFFD4C0EEFFD5C0EEFFAF
:103F1000D6C0EEFFD7C0EEFFD8C0EEFFD9C0EEFF8F
:103F2000DAC0EEFFDBC0EEFFDCC0EEFFDDC0EEFF6F
:103F3000DEC0EEFFDFC0EEFF40D0E0C0EEFFE1C02C
:103F4000EEFFE2C0EEFFE3C0EEFFE4C0EEFFE5C02F
:103F5000EEFFE6C0EEFFE7C0EEFFE8C0EEFFE9C00F
:103F6000EEFFEAC0EEFFEBC0EEFFECC0EEFFEDC0EF
:103F7000EEFFEEC0EEFFEFC0EEFFF0C0EEFFF1C0CF
:103F8000EEFFF2C0EEFFF3C0EEFFF4C0EEFFF5C0AF
:103F9000EEFFF6C0EEFFF7C0EEFFF8C0EEFFF9C08F
:103FA000EEFFFAC0EEFFFBC0EEFFFCC0EEFFFDC06F
:103FB000EEFFFEC0EEFFFFC0EEFF04C0EAFF05C04B
:103FC000E9FF1200F2B4120016500F0AD8B4120022
:103FD000FF0EE3CF0AF0FE0EE3CF0BF0FD0EE3CFB2
:103FE0000CF0FC0EE3CF0DF00A2A16A08D8E0B2AE2
:103FF00016A28F800C2A16A48F860D2A16A68F88EB
:104000000E6A0F6A106A116A35EC20F00A2E0BEF67
:1040100020F016A08D9E0B2E10EF20F016A28F9090
:104020000C2E15EF20F016A48F9600000D2E1BEF1E
:1040300020F016A68F9800000E2E20EF20F0129090
:1040400000000F2E25EF20F012920000102E2AEF14
:1040500020F012940000112E2FEF20F0129657EC52
:1040600020F0133E06EF20F01200D70E136E000072
:104070000000000000004DEC20F0132E37EF20F080
:10408000D70E136E00000000000000004DEC20F081
:10409000132E42EF20F000001200000050EF20F03D
:1040A0000000000000000000000000001200030EED
:0C40B000146E0000142E59EF20F01200D6
:0440BC00150EAF6EC0
:1040C000AC849D9A9D98AC98AC9E948EAB9CAB961C
:1040D000AB8AAB889F9A9D8A0101FE69FF69949C17
:1040E000AC9CAC969F989D88AC8AAB8E1200150E46
:1040F0006F6E6C84A39AA3986C986C9E98846B9C4A
:104100006B966B8A6B88A59AA38A0101FE69FF6989
:1041100098926C9C6C96A598A3886C8A6B8E120002
:10412000D9CFE6FFE1CFD9FFE6529D9AEAC1DFFF82
:104130009D8ADF5000D0E552E552E7CFD9FF12004B
:10414000D9CFE6FFE1CFD9FFE652A39AF6C1DFFF50
:10415000A38ADF5000D0E552E552E7CFD9FF120025
:10416000D9CFE6FFE1CFD9FFE6520101E75103E0E5
:10417000000E17D016D0E851EA6A000FE96E020E61
:10418000EA22EFCFDFFFEA07E82B1F0EE8179D9A20
:10419000E951E85D02E1010EE76F9D8AE66BDF50B1
:1041A00000D0E552E552E7CFD9FF1200D9CFE6FFA4
:1041B000E1CFD9FFE6520101F35103E0000E17D021
:1041C00016D0F451EA6A400FE96E020EEA22EFCFF0
:1041D000DFFFF607F42B1F0EF417A39AF551F45DD9
:1041E00002E1010EF36FA38AF26BDF5000D0E552BB
:1041F000E552E7CFD9FF1200D9CFE6FFE1CFD9FFD3
:104200000101ED5101E0FCD7F051EA6A200FE96E9F
:10421000020EEA22FE0EDBCFEFFFF12BF02B1F0E7A
:10422000F0179D98F051EF5D02E1010EED6F9D8852
:10423000EE6BE552E7CFD9FF1200D9CFE6FFE1CF11
:10424000D9FF0101F95101E0FCD7FC51EA6A600F86
:10425000E96E020EEA22FE0EDBCFEFFFFD2BFC2BF8
:104260001F0EFC17A398FC51FB5D02E1010EF96FD4
:10427000A388FA6BE552E7CFD9FF12000101E6519E
:1042800002E09D9A19D0E951EA6A000FE96E020E28
:10429000EA22AECFEFFFABA203D0AB98AB88EB2BFB
:1042A000ABB4EC2BEA2BE92B1F0EE917E951E85DC3
:1042B00002E1010EE66FE76B12000101F25102E02C
:1042C000A39A19D0F551EA6A400FE96E020EEA226C
:1042D0006ECFEFFF6BA203D06B986B88F72B6BB49C
:1042E000F82BF62BF52B1F0EF517F551F45D02E1B7
:1042F000010EF26FF36B12000101EE5102E09D9886
:1043000012D0EF51EA6A200FE96E020EEA22EF5056
:10431000AD6EF107EF2B1F0EEF17F051EF5D02E1CD
:10432000010EEE6FED6B12000101FA5102E0A3984D
:1043300012D0FB51EA6A600FE96E020EEA22EF50DA
:104340006D6EFD07FB2B1F0EFB17FC51FB5D02E1A1
:10435000010EFA6FF96B1200D9CFE6FFE1CFD9FF5A
:104360000101E55101E110D0E50506E1FE0EDBCFCC
:10437000E6FF42DFE55208D0020EE55D05E1FE0EE4
:10438000DBCFE6FF5ADFE552E552E7CFD9FF120057
:10439000D9CFE6FFE1CFD9FF040EE126FB0EDBCF3C
:1043A0002BF0FC0EDBCF2CF0FD0EDBCF2DF0FE0E44
:1043B000DBCF2EF0C20E206E216A226A236A2BC048
:1043C0001BF02CC01CF02DC01DF02EC01EF078EC90
:1043D00028F017C02BF018C02CF019C02DF01AC00F
:1043E0002EF0F70EDBCF2FF0F80EDBCF30F0F90E0A
:1043F000DBCF31F0FA0EDBCF32F03E0E206E2168BB
:10440000226823682FC01BF030C01CF031C01DF0A3
:1044100032C01EF078EC28F017C02FF018C030F032
:1044200019C031F01AC032F02F502B2630502C22F8
:1044300031502D2232502E222BC0DFFF010E2CC016
:10444000DBFF020E2DC0DBFF030E2EC0DBFFD9CF3A
:10445000E9FFDACFEAFFEECF1BF0EECF1CF0EECF94
:104460001DF0EFCF1EF0D00E206E070E216E226AD7
:10447000236A4FEC25F01BC0DEFF1CC0DEFF1DC011
:10448000DEFF1EC0DDFFDD52DD52DECF1BF0DECFD2
:104490001CF0DECF1DF0DDCF1EF0DD52DD5200D06E
:1044A000D9CFE1FFE552E7CFD9FF1200D9CFE6FF20
:1044B000E1CFD9FF040EE126FB0EDBCF2FF0FC0E7F
:1044C000DBCF30F0FD0EDBCF31F0FE0EDBCF32F074
:1044D000430E206E216A226A236A2FC01BF030C06F
:1044E0001CF031C01DF032C01EF078EC28F017C06F
:1044F0002FF018C030F019C031F01AC032F0F70EAA
:10450000DBCF1BF0F80EDBCF1CF0F90EDBCF1DF07C
:10451000FA0EDBCF1EF0BD0E206E216822682368E4
:1045200078EC28F017502F5C2B6E185030582C6EFA
:10453000195031582D6E1A5032582E6E2BC0DFFF95
:10454000010E2CC0DBFF020E2DC0DBFF030E2EC0C0
:10455000DBFFD9CFE9FFDACFEAFFEECF1BF0EECFDA
:104560001CF0EECF1DF0EFCF1EF0E80E206E030E14
:10457000216E226A236A4FEC25F01BC0DEFF1CC0AF
:10458000DEFF1DC0DEFF1EC0DDFFDD52DD52DECFCF
:104590001BF0DECF1CF0DECF1DF0DDCF1EF0DD52B4
:1045A000DD5200D0D9CFE1FFE552E7CFD9FF1200AD
:1045B0009EB802D0FDD7FCD71200D9CFE6FFE1CFDD
:1045C000D9FFFE0EDBCFE6FFA5EC1EF0E5520D0E87
:1045D000AD6EEEDFE552E7CFD9FF1200D9CFE6FF8F
:1045E000E1CFD9FF0201D950FD0FEC6FFF0EDA20A9
:1045F000ED6F010EEA6AEC25E96EED51EA22EF500B
:10460000E66EA5EC1EF0E552ECC2E9FFEDC2EAFF52
:10461000EF50E66EA5EC1EF0E5520D0EAD6EC8DF54
:10462000E552E7CFD9FF1200D9CFE6FFE1CFD9FF9E
:104630000201EE6B1A0EEE5D11E2FD0EDBCFE9FF1B
:10464000DB2AFE0EDBCFEAFF01E3DB2AEF50E66E4A
:10465000A5EC1EF0E5520201EE2BECD70D0EAD6E6F
:10466000A7DFE552E7CFD9FF12000201A00EEC6FE1
:10467000020EED6F0201A0510201F06FF16BF251D9
:10468000F01902E1F351F11918E00201C0A502D0BE
:10469000C0950FD0F2C2E6FFA5EC1EF0E552F0C2C5
:1046A000E6FFA5EC1EF0E5520D0EAD6E81DF0201B6
:1046B000C095F0C2F2F2F1C2F3F20201F22B000E49
:1046C000F323F33504E2F251FF08000EF35502E242
:1046D000F26BF36B1200150EE66E3C0EE66E49ECC3
:1046E00029F0E552E552320EE66E45EC2AF0E5522D
:1046F0001200D9CFE6FFE1CFD9FFFE0EDBCFEFF2FC
:10470000E552E7CFD9FF1200D9CFE6FFE1CFD9FFBD
:10471000020EE1260F0EE66EFE0EDB507F0BFE0B47
:10472000FD0BE66EF10EE66EB0EC28F0E552E552B8
:10473000E5520A0EE66E63EC2AF0E5527AEC2AF0B6
:1047400007EC04F0000901E0FBD7C5EC29F077EC99
:104750002AF0C4502D6E2DC02EF02D6AC3500001DA
:104760002D102B6E2EC02CF02BC0DEFF2CC0DDFFD9
:10477000DECF2BF0DDCF2CF02BC0F3FF2CC0F4FFED
:0E47800000D0D9CFE1FFE552E7CFD9FF1200FC
:02478E00D9CF81
:10479000E6FFE1CFD9FF020EE126FD0EDBCF2DF0C3
:1047A000FE0EDBCF2EF0FB0EDBCFE9FFFC0EDBCFE6
:1047B000EAFFEE502D5C2B6EEE502E582C6E2BC067
:1047C000DEFF2CC0DDFFDECF2BF0DDCF2CF0F90EAD
:1047D000DBCF2DF0FA0EDBCF2EF02E502C18E8AEEA
:1047E00002D02C3404D02B502D5C2C502E5806E2D5
:1047F000F90EDBCFDEFFDBCFDDFF27D0DECF2BF0E6
:10480000DDCF2CF0F90EDBCF2DF0FA0EDBCF2EF042
:104810002D6C2E1E000E2E222C502E18E8AE02D02B
:104820002E3404D02D502B5C2E502C580EE21D68D7
:104830001E68F90EDBCF22F0FA0EDBCF23F083ECFB
:1048400025F01BC0DEFF1CC0DDFFDECF2BF0DDCF6F
:104850002CF0FB0EDBCFE9FFFC0EDBCFEAFF2B5089
:10486000EE262C50ED22FB0EDBCFE9FFFC0EDBCF5A
:10487000EAFFEECF2BF0EFCF2CF0D8802C5004E7DE
:10488000800E2B5CFF0E2C580AE2FB0EDBCFE9FFFB
:10489000FC0EDBCFEAFF800EEE6EED681AD0FB0E49
:1048A000DBCFE9FFFC0EDBCFEAFFEECF2BF0EFCF43
:1048B0002CF02C3404E22B507F08000E2C5409E21B
:1048C000FB0EDBCFE9FFFC0EDBCFEAFF7F0EEE6EC7
:1048D000ED6AFB0EDBCFE9FFFC0EDBCFEAFFEECF8C
:1048E0002BF0EFCF2CF02BC0F3FF2CC0F4FF00D047
:0C48F000D9CFE1FFE552E7CFD9FF12005D
:0448FC00D9CFE6FF2B
:10490000E1CFD9FF040EE126FB0EDBCF1BF0FC0E3E
:10491000DBCF1CF01D6A1E6A1CAE02D01D681E682B
:104920000A0E206E216A226A236A78EC28F017C0EA
:10493000DEFF18C0DEFF19C0DEFF1AC0DDFFDD524A
:10494000DD52D9CFE9FFDACFEAFFEECF2BF0EECF81
:104950002CF0EECF2DF0EFCF2EF0060E206E010ED4
:10496000216E226A236A2BC01BF02CC01CF02DC0C4
:104970001DF02EC01EF04FEC25F01BC02BF01CC00C
:104980002CF01DC02DF01EC02EF0FD0EDBCFE9FF78
:10499000FE0EDBCFEAFF2BC0EEFF2CC0EDFFD9CF20
:1049A000E1FFE552E7CFD9FF1200D9CFE6FFE1CF13
:1049B000D9FFFD0EDBCFE9FFFE0EDBCFEAFFEECF26
:1049C0002BF0EFCF2CF02C3404E22B500008000E1B
:1049D0002C5409E2FD0EDBCFE9FFFE0EDBCFEAFF30
:1049E000EE06000EEF5AFD0EDBCFE9FFFE0EDBCF29
:1049F000EAFFEECF2BF0EFCF2CF02C3404E22B505B
:104A00000008000E2C5402E2000E01D0010E00D06E
:104A1000E552E7CFD9FF1200D9CFE6FFE1CFD9FFAA
:104A2000FD0EDBCFE9FFFE0EDBCFEAFFEECF2BF072
:104A3000EFCF2CF02C3404E22B500008000E2C5445
:104A400002E2000E01D0010E00D0E552E7CFD9FFFF
:024A5000120052
:0E4A5200256A23AE32EF25F0226C231EE86A9F
:104A60002322251E1EAE3AEF25F01D6C1E1EE86A9D
:104A70001E22251EE4EC29F01EBE4AEF25F025AECD
:104A8000000C1D6C1E1EE86A1E22196C1A1EE86AB4
:104A90001A22000C25BE41EF25F02688FF0C256A5E
:104AA000E86A23AE5CEF25F0206C211E221E231E37
:104AB000212222222322251E1EAE67EF25F01B6C29
:104AC0001C1E1D1E1E1E1C221D221E22251EA1ECA8
:104AD00029F01EBE7EEF25F025AE000C1B6C1C1EBF
:104AE0001D1E1E1EE86A1C221D221E22176C181E87
:104AF000191E1A1E182219221A22000C25BE6EEF4A
:104B000025F02688FF0C1EC02AF01DC029F01D507C
:104B10002202F4CF1CF0F3CF1BF01E502302F4CF7F
:104B20001EF0F3CF1DF02202F3501C26F4501D227C
:104B3000E86A1E2229502302F3501C26F4501D223D
:104B4000E86A1E2223AEA9EF25F029501D5E2A50E7
:104B50001E5A2AAE000C22501D5E23501E5A000C15
:104B60009384F09EF188F092F0889386F186F09419
:104B7000F08A1200D9CFE6FFE1CFD9FF040EE1267B
:104B8000F098E3C2DFFF010EE4C2DBFF020EE5C2D4
:104B9000DBFF030EE6C2DBFFF088DECF1BF0DECFCB
:104BA0001CF0DECF1DF0DDCF1EF0DD52DD5200D057
:104BB000D9CFE1FFE552E7CFD9FF1200F09802010B
:104BC000E36BE46BE56BE66BF088120088B207D00C
:104BD0000201E307000EE45BE55BE65B06D0020141
:104BE000E32B000EE423E523E6231200D9CFE6FFF2
:104BF000E1CFD9FF040EE126F09AE7C2DFFF010EF4
:104C0000E8C2DBFF020EE9C2DBFF030EEAC2DBFFF4
:104C1000F08ADECF1BF0DECF1CF0DECF1DF0DDCF43
:104C20001EF0DD52DD5200D0D9CFE1FFE552E7CFD3
:104C3000D9FF1200F09A0201E76BE86BE96BEA6BAF
:104C4000F08A120088B407D00201E707000EE85B83
:104C5000E95BEA5B06D00201E72B000EE823E923BB
:044C6000EA23120031
:0C4C6400D9CFE6FFE1CFD9FF040EE12616
:104C7000FD0EDBCFE9FFFE0EDBCFEAFF020EEECF2B
:104C8000DBFF030EEDCFDBFFFA0EDB5002E0800E00
:104C900001D0000E2B6E030EDB50400B2B10DF6E8D
:104CA000030EDB503F0BE76E010EE7CFDBFFDF505B
:104CB000400A1BE0C00A19E0800A03E0C00A01E0D4
:104CC00017D0FB0EDB28F36E010EDB50F35C01E125
:104CD0000BD0FB0EDB50F36E010EDB50F35C02E1F8
:104CE000020EDB2A010EDB2A03D0010EDB6A00D0A4
:104CF000FC0EDB50F36E020EDBCFF4FFF350F45CDE
:104D000002E3020EDB6A010EDBCFE6FFFA0EDB5098
:104D100002E0400E01D0000EE552E710E76E030EF0
:104D2000E7CFDBFFFD0EDBCFE9FFFE0EDBCFEAFFB7
:104D3000020EDBCFEEFF030EDBCFEDFF020EDB50EA
:0E4D400000D0D9CFE1FFE552E7CFD9FF120036
:024D4E00D9CFBB
:104D5000E6FFE1CFD9FF040EE126FC0EDB507F0F0A
:104D60002F6E306A316A326AFD0EDBCF2BF0FE0EF9
:104D7000DBCF2CF02D6A2E6A2CAE02D02D682E6867
:104D80002BC01BF02CC01CF02DC01DF02EC01EF03F
:104D90002FC020F030C021F031C022F032C023F00B
:104DA00078EC28F017C0DEFF18C0DEFF19C0DEFF68
:104DB0001AC0DDFFDD52DD52D9CFE9FFDACFEAFFBD
:104DC000EECF1BF0EECF1CF0EECF1DF0EFCF1EF0BC
:104DD0007E0E206E010E216E226A236A4FEC25F0B2
:104DE0001BC0DEFF1CC0DEFF1DC0DEFF1EC0DDFFDE
:104DF000DD52DD52DFCF2BF0010EDBCF2CF02BC0CC
:104E0000F3FF2CC0F4FF00D0D9CFE1FFE552E7CF8C
:044E1000D9FF1200B4
:0C4E14001E0EF66E080EF76E000EF86E13
:104E200002010900F550DE6F0900F550DF6F03E164
:104E3000DE6701D03DD00900F550D96F0900F5506B
:104E4000DA6F0900F550DB6F09000900F550E96ED3
:104E50000900F550EA6E090009000900F550DC6F01
:104E60000900F550DD6F09000900F6CFE0F2F7CF39
:104E7000E1F2F8CFE2F2D9C2F6FFDAC2F7FFDBC205
:104E8000F8FF0201DC5302E1DD5307E00900F550B1
:104E9000EE6EDC07F8E2DD07F9D7E0C2F6FFE1C20B
:104EA000F7FFE2C2F8FF0201DE07000EDF5BBFD7AB
:024EB0001200EE
:0E4EB200FB0EE3CFF6FFFC0EE3CFF7FFFD0E85
:104EC000E3CFF8FFFE0EE3CFE9FFFF0EE3CFEAFFEB
:104ED000E9CFF3FFEACFF4FF0900F5CFEFFFEE666D
:104EE000FBD71200FE0EE3CFE9FFFF0EE3CFEAFF90
:104EF000F36AF46AEE5203E0F34AF42AFBD7120095
:104F0000FF0EE3CFF8FFE552FF0EE3CFF7FFE552C8
:104F1000FF0EE3CFF6FFE552E66AE66AE66A0900AD
:104F2000F55209E0FD0EE32A05E1FE0EE32A02E157
:104F3000FF0EE32AF4D7FD0EE3CF1CF0FE0EE3CF05
:0A4F40001DF0FF0EE3CF1EF012007B
:064F4A00D9CFE6FFDACF2B
:104F5000E6FFE1CFD9FFE2CFDAFFE652E652E652B2
:104F6000E652D950FB0F2B6EFF0EDA202C6E2BC0B1
:104F7000DEFFDD6EDECFE6FFDDCFE6FFFB0EDBCF33
:104F8000E6FFFC0EDBCFE6FFFD0EDBCFE6FFFEC14A
:104F9000E6FFFFC1E6FF4AEC04F0F56E070EE15CA8
:104FA00002E2E16AE552E16EF550020EF3CFDBFF5B
:104FB000030EF4CFDBFF020EDBCF2BF0030EDBCFB3
:104FC0002CF02BC0F3FF2CC0F4FFD9CFE1FFDACFD8
:0E4FD000E2FFE552E5CFDAFFE7CFD9FF12008E
:024FDE00D9CF29
:104FE000E6FFE1CFD9FFFD0EDBCFE9FFFE0EDBCF01
:104FF000EAFF7F0EEF6EFB0EDBCF2BF0FC0EDBCF5C
:10500000E6FFFA0EDB50E552E75CD8802B540CE348
:10501000FD0EDBCFE9FFFE0EDBCFEAFFF90EDBCFA3
:10502000EFFFF36AF46A1ED0FA0EDBCFE6FFFC0E48
:10503000DB50E552E724F36EFB0EDBCFF4FFF350B9
:10504000F45C0CE3FD0EDBCFE9FFFE0EDBCFEAFFE5
:10505000F80EDBCFEFFFF36AF46A04D0010EF36EB3
:0C506000F46A00D0E552E7CFD9FF12003F
:04506C00D9CFE6FFB3
:10507000DACFE6FFE1CFD9FFE2CFDAFFFB0EDBCFDD
:105080002BF0FC0EDBCF2CF00001800E2C141AE16B
:10509000FB0EDBCFE9FFFC0EDBCFEAFFEECFF3FF29
:1050A000EDCFF4FFEE2A000EEF22F3CFE9FFF4CFAD
:1050B000EAFFFD0EDBCFEFFFEF502C6AF36E2CC042
:1050C000F4FF10D0FB0EDB50FE0806E1FD0EDBCF37
:1050D000E6FF55EC2AF005D0FD0EDBCFE6FFACEC89
:1050E00021F0E552E552E5CFDAFFE7CFD9FF120014
:1050F0001B502002F3CF17F0F4CF18F02102F35029
:105100001826000EF420196E1B502202F3501926A7
:10511000000EF4201A6E1B502302F3501A261C5066
:105120002002F3501826F4501922000E1A221C50A7
:105130002102F3501926F4501A221C502202F35077
:105140001A261D502002F3501926F4501A221D5021
:105150002102F3501A261E502002F3501A26120084
:10516000D9CFE6FFDACFE6FFE1CFD9FFE2CFDAFF12
:10517000C26AC16AC06AFC0EDB407F0B3C0BC26E88
:10518000FB0EDB50C16EFC0EDB38F00B300BC11296
:10519000FD0EDB50800BC06EFD0EDB380F0B070BD6
:1051A000C012FD0EDB50040DF350380BC012FC0E84
:1051B000DBAE03D09E9C9D8CF28CC280E552E5CF85
:0851C000DAFFE7CFD9FF12006E
:0851C800D9CFE6FFDACFE6FFC4
:1051D000E1CFD9FFE2CFDAFF3F0EC716C66AFD0E58
:1051E000DB50C612FB0EDB50C712FC0EDB50030A6D
:1051F00009E0010A04E0020A06E1C78C04D0C78C6A
:10520000C68801D0C688FD0EDB50050A03E0010AFE
:1052100004E1978E9486C79E01D09496949A9488C0
:0E522000C68AE552E5CFDAFFE7CFD9FF1200CC
:02522E00D9CFD6
:10523000E6FFDACFE6FFE1CFD9FFE2CFDAFF6C6A13
:105240006B6AFD0EDBB06C88DBA202D06C8C6B8CC1
:10525000DBB46C8EDBA602D06B8801D06B8ADBA836
:1052600002D06C8401D06C94DBAC02D0A38A01D054
:10527000A39ADBAE02D0A38801D0A398FC0EDB502A
:105280006F6E6C8A6B8EE552E5CFDAFFE7CFD9FF00
:0252900012000A
:0E529200D9CFE6FFDACFE6FFE1CFD9FFE2CFBA
:1052A000DAFFAC6AAB6AFD0EDBB0AC88DBA202D0E1
:1052B000AC8CAB8CDBB4AC8EDBA602D0AB8801D05F
:1052C000AB8ADBA802D0AC8401D0AC94DBAC02D0BA
:1052D0009D8A01D09D9ADBAE02D09D8801D09D9819
:1052E000FC0EDB50AF6EAC8AAB8EE552E5CFDAFF39
:0652F000E7CFD9FF120018
:0A52F600D9CFE6FFE1CFD9FFFD0E8E
:10530000DBCF2BF0FE0EDBCF2CF0800E2B2400D059
:10531000E552E7CFD9FF1200D9CFE6FFE1CFD9FFA1
:10532000FE0EDB502B6E2C6A800E2B5E000E2C5A6C
:105330002BC0F3FF2CC0F4FF00D0E552E7CFD9FF1C
:02534000120059
:0E5342001A6A196A186A176A200EE76ED89068
:105350001B361C361D361E361736183619361A36C9
:105360002050175C215018582250195823501A58B1
:1053700009E32050175E2150185A2250195A235021
:0A5380001A5A1B2AE72EE4D7120088
:06538A00D9CFE6FFDACFE7
:10539000E6FFE1CFD9FFE2CFDAFFE652E652C35093
:1053A000DF6E010EC4CFDBFFDECF2BF0DDCF2CF0A4
:1053B0002BC0F3FF2CC0F4FFE552E552E552E5CFD8
:0853C000DAFFE7CFD9FF12006C
:0853C8001A6A196A100EE76E63
:1053D000D8901D361E3619361A362250195C2350C5
:1053E0001A5805E32250195E23501A5A1D2AE72E37
:0453F000F0D71200E0
:0C53F400494649203230303620557365A0
:10540000722050726F636573736F7220496E697496
:0D54100069616C697A6564202E2E2E0D00F6
:02541E002CEC74
:1054200018F071EC13F00201C0910201C0A107D085
:10543000F9EC13F00201A1AD02D062EC0FF070ECB8
:0654400013F0F3D7120087
:0A544600F36AF46AFF0EE124E96E38
:10545000FF0EE220EA6EED6607D02F0EEF6404D057
:0A5460003A0EEF6001D0F32A1200AB
:06546A001EEE00F02EEE24
:1054700000F0F86A269CA68EA69C93EC1EF00AEC1F
:0A54800027F00FEC2AF0F9D7120014
:06548A00FF0EE350336E3B
:10549000480E01D04C0EE76EE72EFED7E76AE72EE6
:0A54A000FED7332EF7D700001200EC
:0654AA00FF0EE350ACBA56
:1054B00004D0AF6AAB8EAC8A949CACA2FED7AD6E22
:0654C000F36EF46A120015
:0A54C600FF0EE350E84E1200000054
:0C54D00000D000D000D0E82EFAD7120067
:0454DC003031323306
:0D54E0003435363738396162636465660023
:0254EE00C2906A
:0454F0009D9C12006D
:0454F400C28212005E
:0854F8000000000000020202A6
:03550000020200A4
:0D5503000000010000000000000100000099
:0C5510000001000000000000010000008D
:02551C0002008B
:02551E0000008B
:02552000000089
:095522000000000000000000FF81
:020000040030CA
:0E000000FF36F6FEFFFF8BFFFFBFFF9FFFBF27
:00000001FF
